:020000040000FA
:02000000D02806
:080008008312B920B920810127
:100010000B11A00A0F302002031D54288312860AF8
:10002000A001A10AC7306B2130302107BE20772103
:100030000A302102031D5428A101A20AC6306B21F7
:1000400030302207C720772106302202031D5428B2
:10005000A201A30AC4306B2130302307BE207721D0
:100060000A302302031D5428A301A40AC3306B21C4
:1000700030302407C720772106302402031D54287E
:10008000A401A50AC1306B2130302507BE2077219D
:100090000A302502031D5428A501A60AC0306B2191
:1000A00030302607772154288B160900A001A101C2
:1000B000A201A301A401A501A601080004302502A4
:1000C000031D080002302602031D080056203421BB
:1000D00008000730C50026308400C50B71280510C4
:1000E00008000008C4001D3084070008C402031D76
:1000F00008001D30840284036D280730C5002630B7
:100100008400C50B8528051008000008C4002D30A8
:1001100084070008C402031D08002D3084028403F4
:1001200081280730C50026308400C50B99280514A6
:1001300008000008C400173084070008C402031D2B
:10014000080017308402840395280730C500263044
:100150008400C50BAD28051408000008C400273032
:1001600084070008C402031D0800273084028403AA
:10017000A928BB30A800A80BBB280800A7003A306C
:100180002702031DC5283030080027080800A700F3
:1001900036302702031DCE2830300800270808001B
:1001A00007309F0083169F01003086008500831270
:1001B0000510831238306B2101306B2103306B2125
:1001C0000F306B2180306B21432221308400342199
:1001D00093219321ED213830840034219321932100
:1001E00083163830840000309B00212318224830C9
:1001F00084003421932193218316483084001030E9
:100200009B002123831297213E30840034219321C7
:10021000932183163E30840007309B0021238312F4
:10022000C2214E30840034219321932183164E3015
:10023000840017309B002123831260212130840029
:1002400034210730831681008312051086010030A7
:1002500081008B178B1686015E208B129120A520C2
:1002600069207D208B162C29C7306B213030000788
:100270007721C6306B21840A303000077721C530E2
:100280006B213A307721C4306B21840A303000076B
:100290007721C3306B21840A303000077721C230C8
:1002A0006B213A307721C1306B21840A303000074E
:1002B0007721C0306B21840A303000077721080095
:1002C00080306B21483077214F30772152307721B1
:1002D0004130772108008600832105158510832190
:1002E00005118510832105158510832108008600DE
:1002F0008321051585148321051185148321051596
:100300008514832108001930AA00A900A90B8629A9
:10031000AA0B85290800FA30AA00A900A90B8E298A
:10032000AA0B8D2908008B218B218B2108008312B9
:1003300038306B2101306B2103306B210F306B2182
:1003400080306B214430772145307721533077213D
:10035000313077213A307721C0306B210630B70039
:10036000433084006622C500463C031DC029450871
:1003700083163E30840007309B002B238312080035
:1003800045080800831238306B2101306B2103309F
:100390006B210F306B2180306B2144307721453049
:1003A000772153307721323077213A307721C030AE
:1003B0006B210630B700533084006622C500463CEE
:1003C000031DEB29450883164E30840017309B002F
:1003D0002B238312080045080800831238306B2154
:1003E00001306B2103306B210F306B2180306B218A
:1003F00041307721433077215430772131307721D4
:100400003A307721C0306B210630B7003D30840090
:100410006622C500463C031D162A4508831638305F
:10042000840000309B002B2383120800450808003D
:10043000831238306B2101306B2103306B210F3078
:100440006B2180306B21413077214330772154304C
:100450007721323077213A307721C0306B21063056
:10046000B7004D3084006622C500463C031D412A7A
:10047000450883164830840010309B002B238312DC
:10048000080045080800831238306B2101306B21C9
:1004900003306B210F306B2180306B21533077217B
:1004A00045307721543077213A307721C0306B21A5
:1004B0000630B700263084006622C500463C031D86
:1004C000642A4508562008004508080003308A00C1
:1004D0008316F030860081138312EF30B00086005F
:1004E0000430B100B00C30088600832106080F38B4
:1004F000B200B209031D7F2AB10B722A6D2A0608C9
:100500000F38B600B609031D7F2A83160030860017
:100510008312B00930080F39B0003208F039B00446
:10052000300886001130B200B203320800233002D6
:10053000031D942A32088600103032070023C500BC
:10054000463C031DA52A4508080045088600B00062
:10055000003083160030860083123008D03E8000C1
:0E056000303E77218403B70B662A93210800F2
:10060000820711341234143418342134223424343F
:10061000283441344234443448348134823484347C
:10062000883430343134323433343434353436343D
:100630003734383439344134423443344434453423
:1006400046340630B70000089A003423840A9B0A17
:10065000B70B232B08000630B70041238000840A23
:100660009B0AB70B2D2B080083161C158B135530D6
:100670009D00AA309D009C149C183C2B1C118B17CC
:0A068000080083161C141A08080075
:02400E00293F48
:00000001FF
